:100000000C9454090C9498090C9498090C94980930
:100010000C9498090C9498090C9498090C949809DC
:100020000C9498090C9498090C94C4140C9496158B
:100030000C9498090C9498090C9498090C949809BC
:100040000C9498090C94172E0C9498090C94980908
:100050000C9498090C941E240C9498090C949809FB
:100060000C9498090C9498090C9498090C9498098C
:100070000C9498090C9498090C9498090C9498097C
:100080000C9498090C9498090C9498090C9498096C
:100090000C9498090C9498090C9498090C9498095C
:1000A0000C9498090C9498090C949809FB151D164A
:1000B00008171D1608175F1682160817D716EA16B6
:1000C000381A381A661A661AA81AE41AE41CE41CCC
:1000D000FC1AE41CF31BF31BBE1CE41CE41CD21C26
:1000E000751901620262016202620035002B00E1B3
:1000F00000E100E00000001E00140004001D0002EA
:10010000304E001F001A0016001B00E300E1002023
:1001100000080007000600AE002C002100150009B1
:1001200000190065744B00220017000A000500004A
:100130000029744C002A0000002800000008544CDC
:10014000002A00000028000000500023001C000BC3
:1001500000110000004F00240018000D001000E600
:1001600000520025000C000E0036002D002C002649
:100170000012000F0037004A00E50027001300338B
:100180000038002E00510030002F00347231724DC3
:1001900071000035002B00E100E100E00000001ECE
:1001A0000034000400330002304E001F00360012FD
:1001B000001400E300E1002000370008000D00AE4D
:1001C000002C002100130018000E0065744B002263
:1001D000001C000C001B00000029744C002A0000C9
:1001E000002800000008544C002A000000280000ED
:1001F000005000230009000700050000004F002404
:10020000000A000B001000E600520025000600174F
:10021000001A002F002C0026001500110019004ABA
:1002200000E50027000F0016001D00300051002ED1
:100230000038002D7231724D710000000000000086
:1002400000000000000000000000000000000000AE
:10025000000000000000000000000000000000009E
:10026000000000000000000000000000000000008E
:10027000000000000000000000000000000000007E
:1006200000000000000000000000000100010001C7
:10063000000100010000003A003F004400010001F9
:100640000001003B00400045000100010001003CAA
:1006500000410001000100010001003D00420001D5
:10066000000100010001003E004300010001000004
:100670000001000100010000000100000001000174
:1006800000010000005000000053003F0001005234
:100690000051000000390040004A004D004F0001A9
:1006A0000001002B005F005C005900620001005453
:1006B0000060005D005A0001300100550061005EDD
:1006C000005B0063000100560057005700580058B7
:1006D00071000001000100010001000100000001A3
:1006E0000001000100010001000100010001000102
:1006F000004C020100010001000100B200490101AB
:1007000000A80001000100B1004902010001000140
:10071000000100B500A800000001004900A9000088
:1007200000AA0000000100490001000000010000D3
:10073000000100B00001000100010000000100A55F
:10074000000100010001000100AC00A60001000151
:1007500000010001000100A70001000100010001EB
:1007600000010046000100010001000100AB00474C
:1007700000480001000100010000000A002530319E
:100780003662003A200025303258000A722F63206A
:1007900030313233343536373839414243444546B7
:1007A0000A000A002530325800626F756E636521B9
:1007B0003A20006C65667420736964652061747406
:1007C00061636865640A006C6566742073696465BA
:1007D000206E6F7420726573706F6E64696E670A45
:1007E00000747279696E6720746F20726573657426
:1007F000206D637032333031380A000A4445425567
:10080000473A20656E61626C65642E0A005B735D19
:10081000004B6579626F6172642073746172742E2B
:100820000A005B575D005B535D005B525D005B44FB
:100830005D005B435D0016034500720067006F00BA
:1008400044006F007800200045005A0000001603A5
:100850004500720067006F0044006F0078002000C0
:1008600045005A0000000403090409028D00050137
:1008700000A0FA090400000103010100092111018F
:100880000001223F000705810308000A0904010056
:100890000103010200092111010001224D00070599
:1008A000820308000A090402000103000000092174
:1008B000110100012236000705830308000A09041C
:1008C00003000203000000092111010001222000A1
:1008D0000705840320000107050403200001090423
:1008E0000400010300000009211101000122390068
:1008F000070585031000011201100100000008ED3A
:10090000FE071301000102000105010906A101050E
:100910000719E029E71500250195087501810205F1
:100920000819012905950575019102950175039135
:1009300001050719002977150025019578750181B2
:1009400002C00631FF0974A1010975150025FF9544
:1009500020750881020976150025FF9520750891FC
:1009600002C005010980A101850216010026B70019
:100970001A01002AB700751095018100C0050C0905
:1009800001A1018503160100269C021A01002A9C80
:1009900002751095018100C005010902A10109013C
:1009A000A100050919012905150025019505750105
:1009B0008102950175038101050109300931158115
:1009C000257F95027508810609381581257F9501D7
:1009D00075088106050C0A38021581257F95017579
:1009E000088106C0C005010906A101050719E02913
:1009F000E7150025019508750181029501750881AB
:100A000001050819012905950575019102950175E2
:100A10000391010507190029FF150025FF950675AB
:100A2000088100C00A002530325820006B657962C9
:100A30006F6172645F7265706F72743A20000A00B1
:100A400025303258006B6579626F6172645F73653F
:100A5000745F6C65643A200064656C5F6B65795FF8
:100A60006269743A2063616E27742064656C3A2071
:100A7000253032580A006164645F6B65795F626992
:100A8000743A2063616E2774206164643A202530D3
:100A900032580A00646F6E652E0A00626F6F676DD0
:100AA00061676963207363616E3A202E2E2E2000E9
:100AB000290A002575002F002575005D2800256492
:100AC000002000256400200025640020002564002B
:100AD0007C0025303258006D6F7573656B65792029
:100AE0005B62746E7C782079207620685D28726560
:100AF000702F61636C293A205B006D6B5F776865CE
:100B0000656C5F74696D655F746F5F6D6178203DC2
:100B10002025640A006D6B5F776865656C5F6D61A9
:100B2000785F7370656564203D2025640A006D6BF5
:100B30005F74696D655F746F5F6D6178203D20251E
:100B4000640A006D6B5F6D61785F7370656564202A
:100B50003D2025640A006D6B5F696E746572766175
:100B60006C203D2025640A006D6B5F64656C6179C3
:100B7000203D2025640A006D6B5F776865656C5FBA
:100B800074696D655F746F5F6D6178203D202564C9
:100B90000A006D6B5F776865656C5F6D61785F7388
:100BA00070656564203D2025640A006D6B5F746983
:100BB0006D655F746F5F6D6178203D2025640A006C
:100BC0006D6B5F6D61785F7370656564203D202596
:100BD000640A006D6B5F696E74657276616C203DAE
:100BE0002025640A006D6B5F64656C6179203D208F
:100BF00025640A000A00257500363A207768656585
:100C00006C5F74696D655F746F5F6D61783A200029
:100C10000A00257500353A20776865656C5F6D615F
:100C2000785F73706565643A20000A0025750034AA
:100C30003A2074696D655F746F5F6D61783A20006A
:100C40000A00257500333A206D61785F7370656521
:100C5000643A20000A00257500323A20696E7465F6
:100C60007276616C286D73293A20000A00257500A0
:100C7000313A2064656C6179282A31306D73293AE4
:100C800020000A092D2056616C756573202D0A001D
:100C90004D3E004D25643E20003F00736574206486
:100CA000656661756C740A00433E20007768657262
:100CB000652064656C74613A20637572736F723D70
:100CC00025642C20776865656C3D25640A5365654D
:100CD00020687474703A2F2F656E2E77696B697077
:100CE000656469612E6F72672F77696B692F4D6F2D
:100CF0007573655F6B6579730A000A092D204D6F66
:100D00007573656B6579202D0A4553432F713A0938
:100D1000717569740A313A0964656C6179282A3100
:100D2000306D73290A323A09696E74657276616CA6
:100D3000286D73290A333A096D61785F73706565B0
:100D4000640A343A0974696D655F746F5F6D617828
:100D50000A353A09776865656C5F6D61785F737015
:100D60006565640A363A09776865656C5F74696D14
:100D7000655F746F5F6D61780A0A703A0970726915
:100D80006E742076616C7565730A643A09736574D4
:100D90002064656661756C74730A75703A092B314D
:100DA0000A646F776E3A092D310A706775703A09D7
:100DB0002B31300A7067646F776E3A092D31300A33
:100DC0000A7370656564203D2064656C7461202A37
:100DD000206D61785F7370656564202A20287265D4
:100DE00070656174202F2074696D655F746F5F6D2D
:100DF0006178290A003F004D3E2000433E20004C10
:100E000025640A000A092D20436F6E736F6C6520FC
:100E10002D0A4553432F713A09717569740A6D3A69
:100E2000096D6F7573656B65790A000A092D204D90
:100E300061676963202D0A643A0964656275670A0F
:100E4000783A096465627567206D61747269780A21
:100E50006B3A096465627567206B6579626F6172D0
:100E6000640A6D3A096465627567206D6F75736514
:100E70000A763A0976657273696F6E0A733A097376
:100E800074617475730A633A09636F6E736F6C658E
:100E9000206D6F64650A302D343A096C6179657292
:100EA000302D34284631302D4634290A506175736F
:100EB0003A09626F6F746C6F616465720A653A0912
:100EC000656570726F6D0A6E3A094E4B524F0A7A21
:100ED0003A09736C656570204C45442074657374E1
:100EE0000A000A002575002E6E6B726F3A20000A08
:100EF000002575002E737761705F6261636B736CA0
:100F00006173685F6261636B73706163653A20004F
:100F10000A002575002E737761705F6772617665D0
:100F20005F6573633A20000A002575002E6E6F5FBF
:100F30006775693A20000A002575002E7377617085
:100F40005F72616C745F726775693A20000A0025F0
:100F500075002E737761705F6C616C745F6C677580
:100F6000693A20000A002575002E636170736C6F6A
:100F7000636B5F746F5F636F6E74726F6C3A2000A7
:100F80000A002575002E737761705F636F6E74724F
:100F90006F6C5F636170736C6F636B3A20000A0063
:100FA00025303258006B65796D61705F636F6E66D6
:100FB00069672E7261773A20000A002575002E6D50
:100FC0006F7573653A20000A002575002E6B6579F0
:100FD000626F6172643A20000A002575002E6D610F
:100FE000747269783A20000A002575002E656E61DA
:100FF000626C653A20000A00253032580064656250
:1010000075675F636F6E6669672E7261773A20005D
:101010000A0025750064656661756C745F6C6179A2
:1010200065723A20003F004E4B524F3A206F666681
:101030000A004E4B524F3A206F6E0A0074696D657C
:10104000725F636F756E743A202530346C580A00F5
:101050006B6579626F6172645F6E6B726F3A2025A7
:10106000580A006B6579626F6172645F69646C65D0
:101070003A2025580A006B6579626F6172645F706F
:10108000726F746F636F6C3A2025580A00686F7333
:10109000745F6B6579626F6172645F6C65647328FD
:1010A000293A2025580A000A092D205374617475C5
:1010B00073202D0A004743433A20342E382E312026
:1010C0004156522D4C4942433A20312E382E30732E
:1010D000766E204156525F415243483A2061767203
:1010E000350A004F5054494F4E533A204C55464113
:1010F00020424F4F544D41474943204D4F55534592
:101100004B45592045585452414B455920434F4E69
:10111000534F4C4520434F4D4D414E44204E4B5272
:101120004F203531320A004255494C443A2035614E
:1011300031386134322D6469727479202831383A3B
:1011400034363A343620466562203231203230312E
:1011500036290A005649443A203078464545442805
:101160004572676F446F7820455A29205049443AA8
:1011700020307831333037284572676F446F7820DC
:10118000455A29205645523A203078303030310ABD
:1011900000444553433A20742E6D2E6B2E206B6510
:1011A00079626F617264206669726D776172652021
:1011B000666F72204572676F646F780A000A092DA6
:1011C0002056657273696F6E202D0A000A6D6F7567
:1011D00073653A206F66660A000A6D6F7573653A2B
:1011E000206F6E0A000A6B6579626F6172643A2043
:1011F0006F66660A000A6B6579626F6172643A20F5
:101200006F6E0A000A6D61747269783A206F6666C3
:101210000A000A6D61747269783A206F6E0A000ADA
:1012200064656275673A206F6E0A000A64656275CC
:10123000673A206F66660A000A0A626F6F746C6F05
:10124000616465722E2E2E2000433E20006565638A
:101250006F6E6669673A0A00536C656570204C458D
:101260004420746573740A00000000000000000050
:10127000000000010204060A0F17202C3A4A5D7193
:10128000879DB3C7DAE9F5FCFFFCF5E9DAC7B39D42
:1012900087715D4A3A2C20170F0A060402010000EC
:1012A000000000000000000011241FBECFEFDAE0B4
:1012B000DEBFCDBF04B603FE24C08091F90190913A
:1012C000FA01A091FB01B091FC018730904BA7403F
:1012D000B04BB9F41092F9011092FA011092FB018F
:1012E0001092FC0114BE84B7877F84BF88E10FB6DB
:1012F000F89480936000109260000FBEE0E0FFE37E
:10130000099511E0A0E0B1E0EAECFFE502C005902C
:101310000D92AA33B107D9F721E0AAE3B1E001C0E9
:101320001D92A93FB207E1F70E94FE110C94E32F32
:101330000C940000FF93EF93E0913A01F0913B0190
:10134000309709F00995EF91FF910895FC0185917F
:10135000803011F0EFDFFBCF0895FF27E0E230E2AD
:1013600047FF0CC0419597FF09C0EDE2609570956D
:1013700080959095611D711D811D911D27FF02C0F3
:10138000219530E350E2AA27660F771F881F991F27
:10139000AA1FA41710F0A41B63955A95A9F7AA30A9
:1013A00008F0A95FA05DAF93F39561157105810504
:1013B000910541F7ED3211F4EF93F395F21718F41C
:1013C0003F93F395FBCF8F91B5DFFA95E1F7089541
:1013D000E991F9918591803021F0853219F0AADFE9
:1013E000F9CF089520E0E89455915532C1F3503378
:1013F00011F4689455915A3348F4505390F3220FE6
:10140000022E220F220F200D250FF4CF0EF421956E
:1014100089919991533619F3533729F1533559F17D
:10142000BC0188279927E8945C3621F48991999129
:1014300068945591543639F446EF7EF077FF0DC02D
:101440008FEF9FEF0AC055374AE039F0583540E139
:1014500021F0523642E009F00895FF93EF937DDFCB
:10146000EF91FF91B7CFFF93EF93FC018191803013
:10147000B9F360DFFBCFFF93EF9368DFF1CFDF932A
:10148000CF93CDB7DEB72596A3DFCF91DF91089537
:10149000613049F0623071F488E00E94BC2189E03B
:1014A0000E94BC2107C0FC018281882319F080EED4
:1014B00090E0089580E090E0089580E090E0089545
:1014C00056985E9825982D9826982E9827982F98AC
:1014D0008091BC019091BD01A091BE01B091BF016E
:1014E00090FF02C0259A2D9A8091C0019091C10170
:1014F000A091C201B091C3010297A105B10511F4F9
:10150000269A2E9A0E94421781FF02C0279A2F9A8C
:1015100080E090E0089580E69AE0892B11F00E9427
:10152000600A80E090E0089556985E9825982D987E
:1015300026982E9827982F988FEF90E09093890007
:101540008093880090938B0080938A0090938D0005
:1015500080938C00259A2D9A2FEF80E792E02150FE
:1015600080409040E1F700C00000269A2E9A2FEFAD
:1015700080E792E0215080409040E1F700C00000F9
:10158000279A2F9A2FEF80E792E0215080409040D9
:10159000E1F700C0000025982D982FEF80E792E03A
:1015A000215080409040E1F700C0000026982E981E
:1015B0002FEF80E792E0215080409040E1F700C09B
:1015C000000027982F9856985E9825982D98269871
:1015D0002E9827982F98089589EA8093800089E0B3
:1015E0008093810024982C983F988AB18F748AB98F
:1015F0006E98479A8BB1806B8BB9769A0E94940A49
:101600008DE59AE0892B11F00E945D0A80E090E060
:10161000089580E28093000180913C0181110EC009
:101620000E94580B81E080933C012FEF83ED90E303
:10163000215080409040E1F700C0000080E40E940B
:101640005E0B8093000181112EC00E94880B809355
:101650000001811128C00E94880B80930001811134
:1016600022C08FE30E94880B8093000181111BC070
:101670000E94800B80E40E945E0B80930001811128
:1016800012C08CE00E94880B8093000181110BC076
:101690000E94880B80930001811105C08FE30E9496
:1016A000880B809300010E94800B809100010895B7
:1016B0001092B9008AE08093B800089594EA90935C
:1016C000BC009091BC0097FFFCCF9091B900987F2F
:1016D000983021F0903111F081E008958093BB00A3
:1016E00084E88093BC008091BC0087FFFCCF809190
:1016F000B900887F883111F0803471F780E0089557
:1017000084E98093BC008091BC0084FDFCCF0895E7
:101710008093BB0084E88093BC008091BC0087FF6D
:10172000FCCF9091B900987F81E0983209F480E075
:10173000089584E88093BC008091BC0087FFFCCFB3
:101740008091BB00089580910001811115C080E453
:101750000E945E0B8093000181110CC082E10E9407
:10176000880B80930001811105C08FEF0E94880BC8
:10177000809300010E94800B84B1807F84B985B181
:10178000807F85B98AB1837F8AB98BB1837F8BB91A
:101790003E98469808950E94090B809300010E948C
:1017A000A30B80B38C7080BB81B3836F81BBECE4EF
:1017B000F1E0AEE3B1E011921D9281E0EA35F80765
:1017C000D1F78CEE9AE0892B11F00C94EC0A089575
:1017D0009F92AF92BF92CF92DF92EF92FF920F93C0
:1017E0001F93CF93DF93809100018823E1F08091D4
:1017F0003D018F5F80933D01811115C081EE97E01F
:101800000E94A6090E94090B80930001882329F0F9
:1018100087EC97E00E94A60906C083EB97E00E9440
:10182000A6090E94940A0EE311E0C0E0D0E0BB24B8
:10183000B39482E0A82ECC24C394D12C24EAE22EC7
:1018400027E0F22EC73000F580910001811162C0BF
:1018500080E40E945E0B80930001811112C082E13E
:101860000E94880B8093000181110BC0C6010C2ED1
:1018700001C0880F0A94EAF780950E94880B809334
:1018800000010E94800B46C0CA30A1F028F4C83085
:1018900059F0C93061F005C0CC3089F070F0CD301E
:1018A00089F0209A289810C0219A29980DC0229A70
:1018B0002A980AC0239A2B9807C0529A01C0539ABB
:1018C0005B9802C03E9A4698E0EAEA95F1F78FB13C
:1018D000799985C092E081708B25892B7C9B02C011
:1018E00090E001C094E0892B7D9B02C090E001C094
:1018F00098E0892B7E9B02C090E001C090E1892B8B
:101900009FB19095991F9927991F9295990F907E55
:10191000892B10C080910001811176C080E40E9463
:101920005E0B80930001882309F45BC0912C0E9418
:10193000800B892DF8019081981739F1808380916F
:101940000101882301F18091D70180FF04C089EA59
:1019500097E00E94A6098091D70180FF0CC080917A
:1019600001011F928F93FF92EF920E943F0A0F9006
:101970000F900F900F908091D70180FF04C082EAF2
:1019800097E00E94A609A09201010E94A30B219654
:101990000F5F1F4FCE30D10509F054CF8091010168
:1019A0008823B1F0815080930101882339F08FE9B9
:1019B0009FE00197F1F700C000000AC0ACE4B1E07D
:1019C000EEE3F1E081918D9391E0EC34F907D1F7EA
:1019D0008BE89AE0892BD1F00E948B0A17C090E027
:1019E0007ACF83E10E94880B8093000181119ECF02
:1019F00081E40E945E0B80930001811197CF0E94C9
:101A0000990B982E909493CF80E094CF81E0DF9152
:101A1000CF911F910F91FF90EF90DF90CF90BF90EB
:101A2000AF909F900895E82FF0E0E45BFE4F808137
:101A30000895CF92DF92EF92FF920F931F93CF936F
:101A4000DF938BE897E00E94A6093CE4E32E31E0A7
:101A5000F32EC0E0D0E046E8C42E47E0D42E0DE7D8
:101A600017E0DF93CF93DF92CF920E943F0A83E883
:101A700097E00E94A609F70181917F0190E00E9402
:101A800087239F938F931F930F930E943F0A8BE7A7
:101A900097E00E94A60921968DB79EB708960FB6CB
:101AA000F8949EBF0FBE8DBFCE30D105D1F6DF9129
:101AB000CF911F910F91FF90EF90DF90CF900895FD
:101AC0008B3B910578F4883A910540F5853A91056C
:101AD000D0F48430910508F0B1C08130910509F44B
:101AE000ADC06BC0803E910508F467C0883E91058B
:101AF00008F4A4C09C01205F31092031310508F0B1
:101B00005CC090650895853A910509F459C0863AFC
:101B1000910509F458C083E890E40895883A910546
:101B200009F454C0893A910509F453C08A3A9105E1
:101B300009F452C08B3A910509F451C08C3A9105D1
:101B400009F450C08D3A910509F44FC0803B9105CE
:101B500009F44EC08E3A910509F44DC08F3A9105B3
:101B600009F44CC0813B910509F44BC0823B9105BF
:101B700009F44AC0833B910509F449C0843B9105AF
:101B800009F448C0853B910509F447C0863B91059F
:101B900009F446C0873B910509F445C0883B91058F
:101BA00009F444C0893B910509F443C08A3B91057F
:101BB00009F042C08AE296E4089580E090E008953A
:101BC00081E890E4089582E890E4089582EE94E438
:101BD000089589EE94E408958AEE94E4089585EBDF
:101BE00094E4089586EB94E4089587EB94E40895D3
:101BF0008CEC94E408958DEC94E4089583E895E4E6
:101C000008958AE895E4089582E995E4089584E9C1
:101C100095E4089581E296E4089583E296E40895B8
:101C200084E296E4089585E296E4089586E296E4D7
:101C3000089587E296E4089580E094E40895089575
:101C400096E0799FF001112494E5899FE00DF11D44
:101C50001124E60FF11DEE0FFF1FE551FF4F859197
:101C600094910895880F991F85599040FC018591A2
:101C700094910895880F991F85519F4FFC0185917C
:101C80009491089526E0729FF001112444E5849F09
:101C9000E00DF11D1124E60FF11DEE0FFF1FE551C0
:101CA000FF4F25913491C9019A9581159F4110F4F8
:101CB000C9010895C90190528115904128F4C901C4
:101CC0009F700E943A0E0895C9019053811590416A
:101CD00020F4C9019927906C0895211580E53807F3
:101CE00069F40E94051D9FEF24E34CE091502040D1
:101CF0004040E1F700C000000C944324213080E50F
:101D0000380751F48BEF97E00E94A6098091D70124
:101D100081608093D7010895C90190558115904144
:101D200008F050C0832F99278F7099278130910533
:101D3000D9F4A9014370552702C0880F991F4A950D
:101D4000E2F79C68A90164E0440F551F6A95E1F72A
:101D500044275370842B952B73E0220F331F7A9501
:101D6000E1F7207633271DC08230910529F4922FA8
:101D70008827816F906A089583309105A9F4A9019D
:101D80004370552781E090E002C0880F991F4A9563
:101D9000E2F79C6843E0220F331F4A95E1F7207E6B
:101DA0003770822B932B08950497F1F4A9014370A7
:101DB000552781E090E002C0880F991F4A95E2F70D
:101DC0009A68E8CFC90190578115904120F4C90164
:101DD0009F7090620895C90190588115904120F438
:101DE000C9019F70906A0895203E3105E0F4203CBF
:101DF000310558F52133310509F470C048F4293212
:101E0000310509F464C02A32310509F46EC074C08A
:101E100029333105F1F022383105D9F02533310568
:101E200009F44EC069C0233E310589F138F4203EE3
:101E30003105C1F0223E3105E1F05EC0263E31059C
:101E400069F1273E3105A9F157C0C9010E94320E40
:101E500008958091EA0180FD02C081FF4DC080EEAF
:101E600090E04BC08091EA0180FFF9CF89E390E0D8
:101E700044C08091EA0182FF0EC08091EA0184FF94
:101E800003C080E090E039C083EE90E036C08091DE
:101E9000EA0182FFF2CF82EE90E02FC08091EA014A
:101EA00083FF0BC08091EA0184FDEBCF87EE90E0C9
:101EB00024C08091EA0183FFF5CF86EE90E01DC03B
:101EC0008091EA0185FF07C089E290E016C0809109
:101ED000EA0185FFF9CF85E390E00FC08091EA0128
:101EE00086FF07C08AE290E008C08091EA0186FF81
:101EF000F9CF81E390E001C0C9010E94600D08950F
:101F0000089580916D0108959FB7F89410925C0137
:101F10009FBF9091F001943009F058C09091E90072
:101F20009F702091EC0020FF02C020E801C020E05B
:101F3000292B94E09093E9009091EB0090FF43C02F
:101F40009091EE0097FF3FC090915A01992321F0A4
:101F50009091E80095FF37C010925A0196E03091B9
:101F6000E80035FD15C03091F001343061F5309155
:101F7000EB0035FD28C0915021F481E080935A0197
:101F800022C0EFE9FFE03197F1F700C00000E7CF92
:101F90008093F1008091E80085FD0AC08091E800FF
:101FA00080FFFCCF8091E8008E778093E80006C028
:101FB0008FB7F89491E090935C018FBF2F702093BE
:101FC000E90080E008952F702093E9008FEF0895D5
:101FD000CF93DF9300D01F92CDB7DEB72091F001F1
:101FE000243019F523E029839B838A832093E90019
:101FF0008FEF9091E800815095FD06C095ED9A9580
:10200000F1F700008111F5CF8091E80085FF0DC048
:1020100040E050E063E070E0CE0101960E94B7120C
:102020008091E8008E778093E8000F900F900F90DA
:10203000DF91CF910895CF93DF9300D01F92CDB75A
:10204000DEB72091F001243021F522E029839B8323
:102050008A8383E08093E9008FEF9091E8008150BC
:1020600095FD06C095ED9A95F1F700008111F5CF29
:102070008091E80085FF0DC040E050E063E070E033
:10208000CE0101960E94B7128091E8008E7780936E
:10209000E8000F900F900F90DF91CF91089520915D
:1020A000F0012430F1F422E02093E9002FEF309189
:1020B000E800215035FD06C035ED3A95F1F70000F6
:1020C0002111F5CF2091E80025FF0BC040E050E042
:1020D00065E070E00E94B7128091E8008E778093EF
:1020E000E8000895CF93DF93EC018091F0018430F4
:1020F00009F047C080910C018823E1F080910D0127
:102100008823C1F085E08093E9008FEF9091E8008B
:10211000815095FD06C095E19A95F1F70000811177
:10212000F5CF8091E80085FF2CC040E050E060E1F1
:1021300070E017C081E08093E9008FEF9091E80094
:10214000815095FD06C095ED9A95F1F7000081113B
:10215000F5CF8091E80085FF14C040E050E068E0D2
:1021600070E0CE010E94B7128091E8008E778093D4
:10217000E80080E1FE01ADE5B1E001900D928A95A5
:10218000E1F7DF91CF91089582E398E00E94A609DC
:102190008091EF01811109C00E9449140E94A61488
:1021A0008091E20084608093E20008958EE298E0DE
:1021B0000E94A6091092EF0108958AE298E00C941B
:1021C000A60986E298E00E94A6090C94042E82E2F9
:1021D00098E00E94A6090E94DE230E940A2E0E9417
:1021E00042170C94800F80915B018F5F80935B019D
:1021F00062E30E94782F911135C010925B018091AB
:102200005C01882379F18091F001843049F5809157
:10221000E9008F709091EC0090FF02C090E801C03F
:1022200090E0982B84E08093E9008091EB0080FFA0
:1022300014C08091EE0087FF10C08091E80085FFF8
:1022400003C01092F100F9CF8091E80080FF05C033
:102250008091E8008E778093E8009F709093E9006A
:1022600010925C01089542E061EC81E00E94C3138A
:1022700042E061EC82E00E94C31342E061EC83E043
:102280000E94C31342E261EC84E00E94C31342E166
:1022900061EC85E00C94C3138091F201833009F462
:1022A00055C030F4813071F0823009F48EC0089549
:1022B0008A3009F47AC08B3009F460C0893009F0A3
:1022C0009CC020C08091F101813A09F096C08091B4
:1022D000E800877F8093E8008091F5019091F601F6
:1022E000892B21F060E080E090E003C060E18DE5A3
:1022F00091E070E00E9400138091E8008B7780935A
:10230000E80008958091F101813209F076C0809152
:10231000F5019091F601009719F0049709F06DC04E
:102320008091E800877F8093E8008091E80082FD3B
:1023300005C08091F0018111F8CF5FC08091F1005C
:1023400080936D018091E8008B7753C08091F101FB
:10235000813A09F052C08091F5019091F601892BE4
:1023600009F04BC08091E800877F8093E80080915E
:10237000E80080FFFCCF80910C0136C08091F10114
:102380008132D9F58091F5019091F601892BA9F55B
:102390008091E800877F8093E8000E94F813809185
:1023A000F30180930C010C94051D8091F1018132A1
:1023B00021F58091E800877F8093E8000E94F81360
:1023C0008091F40180936E0108958091F101813A2A
:1023D000A1F48091E800877F8093E8008091E80075
:1023E00080FFFCCF80916E018093F1008091E80026
:1023F0008E778093E8000C94F813089584B7877F54
:1024000084BF88E10FB6F89480936000109260005A
:102410000FBE90E080E80FB6F8948093610090932F
:1024200061000FBE0E94CB170E9449140E94A6149F
:102430008091E20084608093E20084E89FE00E9443
:10244000702378940E9420170E94CD1782E091E0BB
:102450000E943D170E94F22D81E198E00E94A6099A
:102460008091F001853089F48DE098E00E94A60902
:102470000E94A1238091EE01882391F30E94C92339
:10248000882371F30E94A112EBCF0E94FB17E8CFC3
:10249000292F332723303105A9F06CF42130310581
:1024A00009F442C02230310509F043C08DE890E0C4
:1024B0002AE638E042C021323105C9F02232310526
:1024C00019F137C099278130910541F0823091058B
:1024D00041F0892B71F5E6E6F8E005C0EEE4F8E09E
:1024E00002C0E6E3F8E0849190E09F0126C06530E9
:1024F00000F5E62FF0E0EE0FFF1FEB5DFE4F2081B1
:10250000318189E090E019C0653098F4E62FF0E061
:10251000DF01AA0FBB1FA55EBE4F2D913C91EA5E65
:10252000FE4F808190E009C082E190E027EF38E023
:1025300004C080E090E020E030E0FA0131832083A5
:10254000089580E189BD82E189BD09B400FEFDCF17
:102550008091D8008F7D8093D8008091E0008260C8
:102560008093E0008091E00081FDFCCF0895CF9240
:10257000DF92EF92FF920F931F93CF93DF937C0133
:102580008B01EA010E941914811131C0209731F0AA
:1025900088819981081B190BE80EF91EC12CD12CDA
:1025A0000115110519F18091E80085FD14C0809195
:1025B000E8008E778093E800209741F08881998128
:1025C0008C0D9D1D9983888385E011C00E9419148C
:1025D000882331F30CC0F70181917F018093F100D2
:1025E00001501109FFEFCF1ADF0ADACF80E0DF9147
:1025F000CF911F910F91FF90EF90DF90CF900895B2
:102600002091F7013091F8012617370748F061153E
:10261000710539F42091E8002E772093E80001C07D
:10262000B901FC0120E061157105B9F18091F0015B
:10263000882309F440C0853009F43FC08091E80048
:1026400083FD3DC08091E80082FF06C08091E800D4
:1026500082FF26C080E008958091E80080FFE3CFEC
:102660002091F3008091F20090E0922B61157105AA
:1026700051F08830910538F421912093F100615098
:1026800071090196F3CF21E0089709F020E08091CD
:10269000E8008E778093E800C6CF2111C7CFD6CF50
:1026A0008091F001882339F0853039F08091E8007D
:1026B00083FFCCCF04C082E0089583E0089581E0D9
:1026C00008952091F7013091F8012617370748F057
:1026D0006115710539F42091E8002E772093E80008
:1026E00001C0B901FC0120E061157105C1F18091C3
:1026F000F001882309F441C0853009F440C080917D
:10270000E80083FD3EC08091E80082FF06C0809112
:10271000E80082FF27C080E008958091E80080FFF4
:10272000E3CF2091F3008091F20090E0922B6115AD
:10273000710559F08830910540F424912093F100FF
:102740003196615071090196F2CF21E0089709F0A6
:1027500020E08091E8008E778093E800C5CF2111BA
:10276000C6CFD5CF8091F001882339F0853039F07C
:102770008091E80083FFCBCF04C082E0089583E01E
:10278000089581E00895982F973058F59093E900C7
:10279000981739F07091EC002091ED005091F00005
:1027A00003C0242F762F50E021FF19C03091EB0099
:1027B0003E7F3093EB003091ED003D7F3093ED0094
:1027C0003091EB0031603093EB007093EC0020937C
:1027D000ED005093F0002091EE0027FF07C09F5FAF
:1027E000D3CF8F708093E90081E0089580E0089551
:1027F0008091F10187FD05C08091E80080FF0EC047
:1028000012C08091E80082FD05C08091F001811125
:10281000F8CF08958091E8008B7708C08091F0018F
:102820008111EACF08958091E8008E778093E800C7
:1028300008958091E4009091E50045E62091EC0038
:1028400020FF21C02091E80020FD21C02091F0014F
:10285000222389F0253089F02091EB0025FD0FC05F
:102860002091E4003091E5002817390739F34150F1
:1028700041F0C901E3CF82E0089583E0089581E04B
:10288000089584E008952091E80022FFDFCF80E0E2
:1028900008950E94B7140E94BF14E0EEF0E080811A
:1028A00081608083E8EDF0E080818F77808319BCC0
:1028B000A7EDB0E08C918E7F8C9380818F7E80839A
:1028C0001092EF0108950F931F93CF93DF930E940F
:1028D000B7140E94BF14C8EDD0E088818F77888339
:1028E00088818068888388818F7D888319BC109255
:1028F000F0011092EC011092EE011092ED0100EE49
:1029000010E0F80180818B7F8083888181608883DB
:1029100042E060E080E00E94C313E1EEF0E08081DD
:102920008E7F8083E2EEF0E0808181608083808111
:1029300088608083F80180818E7F808388818061B8
:102940008883DF91CF911F910F910895E8EDF0E01A
:1029500080818F7E8083E7EDF0E0808181608083DD
:1029600084E082BF81E08093EF010C946314E8ED72
:10297000F0E080818E7F80831092E20008951092B3
:10298000DA001092E10008951F920F920FB60F9295
:1029900011242F933F934F935F936F937F938F9364
:1029A0009F93AF93BF93EF93FF938091E10082FFDA
:1029B0000BC08091E20082FF07C08091E1008B7F15
:1029C0008093E1000E94F3108091DA0080FF1FC025
:1029D0008091D80080FF1BC08091DA008E7F8093A9
:1029E000DA008091D90080FF0DC080E189BD82E1CD
:1029F00089BD09B400FEFDCF81E08093F0010E9403
:102A0000C41005C019BC1092F0010E94D61080912C
:102A1000E10080FF19C08091E20080FF15C0809125
:102A2000E2008E7F8093E2008091E20080618093DB
:102A3000E2008091D80080628093D80019BC85E0C4
:102A40008093F0010E94E1108091E10084FF30C08A
:102A50008091E20084FF2CC080E189BD82E189BDC4
:102A600009B400FEFDCF8091D8008F7D8093D800FF
:102A70008091E1008F7E8093E1008091E2008F7E63
:102A80008093E2008091E20081608093E200809177
:102A9000EC01882311F084E007C08091E30087FFF8
:102AA00002C083E001C081E08093F0010E94E71042
:102AB0008091E10083FF29C08091E20083FF25C05F
:102AC0008091E100877F8093E10082E08093F001B4
:102AD0001092EC018091E1008E7F8093E100809163
:102AE000E2008E7F8093E2008091E200806180931B
:102AF000E20042E060E080E00E94C3138091F000B9
:102B000088608093F0000E94DD10FF91EF91BF91EB
:102B1000AF919F918F917F916F915F914F913F9175
:102B20002F910F900FBE0F901F9018951F920F922C
:102B30000FB60F9211242F933F934F935F936F9390
:102B40007F938F939F93AF93BF93CF93EF93FF9315
:102B5000C091E900CF708091EC001092E900809163
:102B6000F000877F8093F00078940E94D215109235
:102B7000E9008091F00088608093F000C093E90044
:102B8000FF91EF91CF91BF91AF919F918F917F91E5
:102B90006F915F914F913F912F910F900FBE0F90CA
:102BA0001F9018951F93CF93DF93CDB7DEB7AA97E9
:102BB0000FB6F894DEBF0FBECDBFE1EFF1E080911C
:102BC000F100819321E0E93FF207C9F70E944C111F
:102BD0008091E80083FF1CC12091F1013091F20146
:102BE000832F90E08A30910508F012C1FC01EA5A67
:102BF000FF4F0C94982F203881F0223809F008C13B
:102C00008091F5018F708093E9008091EB0085FB46
:102C1000882780F91092E90006C08091ED0190911B
:102C2000EE01911182609091E800977F9093E80007
:102C30008093F1001092F100C5C0822F8D7F09F0C2
:102C4000E7C0222319F0223061F0E2C08091F30145
:102C5000813009F0DDC0333009F080E08093EE016F
:102C600028C08091F301811124C02091F5012F70BB
:102C700009F4CEC02093E9008091EB0080FF19C0D9
:102C80008091EB00333011F4806211C08061809339
:102C9000EB0081E090E0022E01C0880F0A94EAF771
:102CA0008093EA001092EA008091EB0088608093A4
:102CB000EB001092E9008091E800877F86C0211127
:102CC000A7C01091F3011F778091E3008078812BDA
:102CD0008093E3008091E800877F8093E8000E9462
:102CE000F8138091E80080FFFCCF8091E3008068BA
:102CF0008093E300112311F083E001C082E0809310
:102D0000F00186C02058223008F082C08091F30183
:102D10009091F4018C3D23E0920779F583E08A835A
:102D20008AE289834FB7F894DE01139620E03EE0F3
:102D300051E2E32FF0E050935700E49120FF03C0ED
:102D4000E295EF703F5FEF708E2F90E0EA3010F069
:102D5000C79601C0C0968D939D932F5F243149F78C
:102D60004FBF8091E800877F8093E8006AE270E0BF
:102D7000CE0101960E94001314C0AE014F5F5F4F59
:102D80006091F5010E944812009709F441C020911A
:102D9000E800277F2093E800BC0189819A810E9486
:102DA00061138091E8008B778093E80031C0203870
:102DB00079F58091E800877F8093E8008091EC01AD
:102DC0008093F1008091E8008E778093E8000E9464
:102DD000F8131EC021111CC09091F3019230C0F471
:102DE0008091E800877F8093E8009093EC010E9437
:102DF000F8138091EC01811104C08091E30087FFFA
:102E000002C084E001C081E08093F0010E94331190
:102E10008091E80083FF0AC08091E800877F80935B
:102E2000E8008091EB0080628093EB00AA960FB6D9
:102E3000F894DEBF0FBECDBFDF91CF911F910895F3
:102E4000CF938091F0018823B1F08091E9008F70D9
:102E50009091EC0090FF02C090E801C090E0C92F73
:102E6000C82B1092E9008091E80083FD0E94D215E2
:102E7000CF70C093E900CF9108959093740180932F
:102E800073010895E0917301F0917401309721F07E
:102E90000190F081E02D099480E00895FF920F9356
:102EA0001F93CF93DF938C01E0917301F091740134
:102EB000309799F10280F381E02D09958091D70137
:102EC00082FF2BC080FF04C08CE29AE00E94A6091A
:102ED000E80180E1F82E06E21AE08091D70180FF38
:102EE0000BC088811F928F931F930F930E943F0AFC
:102EF0000F900F900F900F90FA942196F110EDCF54
:102F00008091D70180FF09C084E29AE0DF91CF91E0
:102F10001F910F91FF900C94A609DF91CF911F9103
:102F20000F91FF900895E0917301F0917401309733
:102F300021F00480F581E02D09940895209171011C
:102F4000309172018217930771F090937201809310
:102F50007101E0917301F0917401309721F00680C6
:102F6000F781E02D0994089520916F01309170014F
:102F70008217930771F09093700180936F01E09135
:102F80007301F0917401309721F00084F185E02DF8
:102F90000994089508950C94CA170E94E0230E9492
:102FA000CB0B0C94A624CF93C82F8091D70182FF1E
:102FB0001EC080FF04C085E49AE00E94A6098091AB
:102FC000D70180FF0CC01F92CF9320E43AE03F93DB
:102FD0002F930E943F0A0F900F900F900F908091B7
:102FE000D70180FF04C08EE39AE00E94A6098C2FCF
:102FF000CF910C94800FCF92DF92EF92FF920F93BC
:103000001F93CF93DF93CDB7DEB72B970FB6F8940E
:10301000DEBF0FBECDBF0E94E80B36E7E32E31E0E6
:10302000F32E00E010E0C02E802F0E94130DF70158
:10303000D1907F01D826B1F40F5F1F4F0E301105DC
:1030400091F78FEF89838A831B820E94E923816035
:10305000782F9D838C8349815A816B818D810E9459
:103060009E1841C09091D70191FF04C08B870E94A8
:10307000190D8B8520E030E04D2D50E0922FBA01E4
:10308000022E02C0759567950A94E2F760FF25C08D
:103090002E83CF82EE24E394F12C02C0EE0CFF1CB1
:1030A0009A95E2F790E08E219F2121E0892B09F487
:1030B00020E028870E94E9238160782F9A878987FA
:1030C0004E815F8168858A850E949E18F801EA58C2
:1030D000FE4F80818E25808306C02F5F3F4F2630B4
:1030E000310561F6A9CF0E941428109175010E9444
:1030F00042171817A1F00E944217809375012B9672
:103100000FB6F894DEBF0FBECDBFDF91CF911F91F8
:103110000F91FF90EF90DF90CF900C94D3172B96E8
:103120000FB6F894DEBF0FBECDBFDF91CF911F91D8
:103130000F91FF90EF90DF90CF900895CF93DF93A2
:10314000CDB7DEB72B970FB6F894DEBF0FBECDBF5D
:103150004F83588769877A878B87DE01119686E0CF
:10316000FD0111928A95E9F785E0FE0137960190FD
:103170000D928A95E1F749815A816B817C818D811D
:103180009E810E94D11F2B960FB6F894DEBF0FBE12
:10319000CDBFDF91CF910895CF93C82F882309F435
:1031A000C1C0823859F40E94421781FDBBC089E337
:1031B0000E946E220E944A2389E30CC0833879F46E
:1031C0000E94421780FDAEC083E50E946E220E94DD
:1031D0004A2383E50E94BF22CF910C944A2384386E
:1031E00059F40E94421782FD9DC087E40E946E221E
:1031F0000E944A2387E4EECF8CEF8C0F813A48F48B
:103200008C2F0E949D2C81118DC08C2F0E946E22CC
:10321000E3CF80E28C0F883048F4C77081E001C0B2
:10322000880FCA95EAF70E941123D6CF8BE58C0F41
:10323000833078F4C53A29F0C63A31F482E890E058
:1032400005C081E890E002C083E890E0CF910C9443
:103250009E1788E58C0F833108F064C0C83A39F1B5
:10326000C93A41F1CA3A49F1CB3A51F1CC3A59F154
:10327000CD3A61F1C03B69F1CE3A71F1CF3A79F1C3
:10328000C13B81F1C23B89F1C33B91F1C43B99F150
:10329000C53BA1F1C63BA9F1C73BB1F1C83BB9F1B0
:1032A000C93BC1F1CA3BC9F58AE292E038C082EE5F
:1032B00090E035C089EE90E032C08AEE90E02FC0F9
:1032C00085EB90E02CC086EB90E029C087EB90E086
:1032D00026C08CEC90E023C08DEC90E020C083E809
:1032E00091E01DC08AE891E01AC082E991E017C020
:1032F00084E991E014C081E292E011C083E292E09F
:103300000EC084E292E00BC085E292E008C086E243
:1033100092E005C087E292E002C080E090E0CF91A9
:103320000C94B417CF910895882309F44BC08238C8
:1033300059F40E94421781FF45C089E30E946E2222
:103340000E944A2389E30CC0833871F40E9442171B
:1033500080FF38C083E50E946E220E944A2383E5E5
:103360000E94BF220C944A23843859F40E944217C9
:1033700082FF28C087E40E946E220E944A2387E4CD
:10338000EFCF9CEF980F913A58F390E2980F983056
:1033900050F4877091E001C0990F8A95EAF7892F60
:1033A0000E941723DFCF9BE5980F933020F480E035
:1033B00090E00C949E17885A833120F480E090E0CE
:1033C0000C94B4170895882321F00E9411230C94C3
:1033D0004A230895882321F00E9417230C944A233E
:1033E0000895CF92DF92EF92FF920F931F93CF93A6
:1033F000DF93CDB7DEB728970FB6F894DEBF0FBEC8
:10340000CDBF8C0185E0F801DE01119601900D928F
:103410008A95E1F7F80140813181F280258122957A
:103420002F7083819481892B31F03F3F31F481E00B
:103430004F3F19F403C081E001C080E080FDC4C2A9
:1034400049833A8389819A812F830E942C229E830B
:1034500088870E942B220E94FE204E81E42FE29555
:10346000EF70F0E0E05AFF4F2F8168850C94982FA1
:10347000842F807F142F1F70882311F01295107FE6
:10348000FF2059F0112309F454C2812F68870E944C
:1034900021230E944A2368854CC2862F0E949419DA
:1034A000112309F491C2812F0E94272328960FB679
:1034B000F894DEBF0FBECDBFDF91CF911F910F916A
:1034C000FF90EF90DF90CF900C944A23342F307F01
:1034D000842F8F70303211F08295807F662319F02F
:1034E000613019F12BC0FF20B1F0222309F493C100
:1034F000213009F090C128960FB6F894DEBF0FBEB8
:10350000CDBFDF91CF911F910F91FF90EF90DF9092
:10351000CF900C943123222319F0213009F454C2A6
:103520008E830E9434238E8189C1FF2021F02230B6
:1035300008F04AC270C1211147C280C1FF2021F0AA
:10354000222309F468C1F5C1222309F477C105C219
:10355000242F26952695237030E02115310521F082
:1035600021303105C9F030C2FF2021F0862F942F81
:10357000937002C080E090E028960FB6F894DEBF0A
:103580000FBECDBFDF91CF911F910F91FF90EF90B4
:10359000DF90CF900C949E17FF2021F0862F942F60
:1035A000937002C080E090E028960FB6F894DEBFDA
:1035B0000FBECDBFDF91CF911F910F91FF90EF9084
:1035C000DF90CF900C94B417862FFF2019F00E9443
:1035D0009A2602C00E94022728960FB6F894DEBFF2
:1035E0000FBECDBFDF91CF911F910F91FF90EF9054
:1035F000DF90CF900C948727842F837009F076C0DA
:10360000F110E2C1262F229526952770220F220F56
:10361000862F8F70C82ED12CE12CF12C022E04C0E5
:10362000CC0CDD1CEE1CFF1C0A94D2F764FF10C00A
:103630006FE070E080E090E004C0660F771F881FA5
:10364000991F2A95D2F7609570958095909503C043
:1036500060E070E0CB01242F269526952370422F41
:1036600050E042305105D1F04330510559F16C29F9
:103670007D298E299F294130510541F128960FB6A9
:10368000F894DEBF0FBECDBFDF91CF911F910F9198
:10369000FF90EF90DF90CF900C9423216C297D292F
:1036A0008E299F2928960FB6F894DEBF0FBECDBF96
:1036B000DF91CF911F910F91FF90EF90DF90CF900E
:1036C0000C943D210E942321C701B60128960FB614
:1036D000F894DEBF0FBECDBFDF91CF911F910F9148
:1036E000FF90EF90DF90CF900C940921FF2019F00C
:1036F000842F817001C08695882309F465C1262F27
:10370000229526952770220F220F862F8F70C82EA4
:10371000D12CE12CF12C022E04C0CC0CDD1CEE1CB3
:10372000FF1C0A94D2F764FF10C06FE070E080E0E5
:1037300090E004C0660F771F881F991F2A95D2F763
:10374000609570958095909503C060E070E0CB0126
:10375000242F269526952370422F50E042305105A4
:10376000D1F04330510559F16C297D298E299F29CB
:103770004130510541F128960FB6F894DEBF0FBED7
:10378000CDBFDF91CF911F910F91FF90EF90DF9010
:10379000CF900C94F7216C297D298E299F2928969A
:1037A0000FB6F894DEBF0FBECDBFDF91CF911F9152
:1037B0000F91FF90EF90DF90CF900C9411220E9418
:1037C000F721C701B60128960FB6F894DEBF0FBEE9
:1037D000CDBFDF91CF911F910F91FF90EF90DF90C0
:1037E000CF900C94DD21603FC9F118F4603E50F495
:1037F0009BC0623F09F460C008F44AC0633F09F40B
:103800006FC092C0162F1F70842F8F71FF2099F008
:103810000E947621812F28960FB6F894DEBF0FBE46
:10382000CDBFDF91CF911F910F91FF90EF90DF906F
:10383000CF900C94E3190E949721812F28960FB600
:10384000F894DEBF0FBECDBFDF91CF911F910F91D6
:10385000FF90EF90DF90CF900C94EA19FF20A1F039
:103860002111B2C0842F8F7128960FB6F894DEBF55
:103870000FBECDBFDF91CF911F910F91FF90EF90C1
:10388000DF90CF900C94BC21223008F09DC0EACF8D
:10389000FF20A1F0842F8F7128960FB6F894DEBF19
:1038A0000FBECDBFDF91CF911F910F91FF90EF9091
:1038B000DF90CF900C947621FF2061F3842F8F71DD
:1038C00028960FB6F894DEBF0FBECDBFDF91CF9123
:1038D0001F910F91FF90EF90DF90CF900C94972164
:1038E000FF2091F0842F8F7128960FB6F894DEBFD9
:1038F0000FBECDBFDF91CF911F910F91FF90EF9041
:10390000DF90CF900C94612128960FB6F894DEBF1B
:103910000FBECDBFDF91CF911F910F91FF90EF9020
:10392000DF90CF900C945721FF20A1F0222309F4BF
:10393000B1CF862F28960FB6F894DEBF0FBECDBF4D
:10394000DF91CF911F910F91FF90EF90DF90CF907B
:103950000C94CC18222309F4B1CF862F28960FB6E9
:10396000F894DEBF0FBECDBFDF91CF911F910F91B5
:10397000FF90EF90DF90CF900C9494194F70C80196
:103980000E94480A28960FB6F894DEBF0FBECDBF3E
:10399000DF91CF911F910F91FF90EF90DF90CF902B
:1039A0000C947E204F70C80128960FB6F894DEBFA5
:1039B0000FBECDBFDF91CF911F910F91FF90EF9080
:1039C000DF90CF900C941F0E28960FB6F894DEBFB0
:1039D0000FBECDBFDF91CF911F910F91FF90EF9060
:1039E000DF90CF9008950E942E230E9403230E940F
:1039F0004A230E94B5280E94872780E090E00E9419
:103A00009E1780E090E00C94B4170E941E230C9443
:103A1000F31C0E942C22292F22952F7030E02C308D
:103A200031054CF42A3031056CF422503109223032
:103A3000310590F407C02C30310551F02F3031059D
:103A400039F00AC0803E10F0803F31F481E00895E3
:103A500093FB882780F9089580E00895CF93DF9342
:103A600000D000D01F92CDB7DEB70F900F900F900F
:103A70000F900F90DF91CF910895CF93DF9300D0F7
:103A800000D000D0CDB7DEB726960FB6F894DEBFD3
:103A90000FBECDBFDF91CF9108951F93CF93DF93DA
:103AA000C091840116E080918501C81799F0D0E09B
:103AB0001C9FF0011D9FF00D1124EA57FE4F40811D
:103AC000518162817381848195810E943D1D21967F
:103AD000C770E9CFDF91CF911F9108954091B60152
:103AE0005091B7016091B8017091B9018091BA010C
:103AF0009091BB010C943D1DCF938091BB018295A9
:103B00008F7009F05FC08091B801882309F45AC012
:103B100020918401A09185016091B6017091B70157
:103B20008091B9019091BA0131E06F3F09F030E026
:103B3000B32FC6E02A1709F445C0009721F07F3F54
:103B400021F44B2F03C041E001C040E030E040FDD4
:103B500035C0C29FF001C39FF00D1124EA57FE4FFC
:103B6000418174132BC04081641328C042814111EC
:103B700025C0438154814817590710F44150510919
:103B8000481B590B483C5105C8F48091BB018F700C
:103B900080618093BB0186E0829FF001839FF00DDE
:103BA0001124E557FE4F80818F708061808386EB02
:103BB00091E00E94F119CF910C944D1D2F5F3F4F62
:103BC0002770B8CFCF910895CF92DF92EF92FF92F6
:103BD0000F931F93CF93DF93CDB7DEB762970FB6E6
:103BE000F894DEBF0FBECDBF8C0185E0F801DE0189
:103BF0001D9601900D928A95E1F7D8014C9111968E
:103C00005C91119712966C9112971396ED90FC901F
:103C100014977091B601E091B7012091B9013091EC
:103C2000BA012115310531F0EF3F31F481E07F3FDA
:103C300019F403C081E001C080E0B82FB170CB2E31
:103C400080FD6CC1D090B801DD2009F4F5C0F09181
:103C5000BB01E216F30638F0C701821B930B883CC8
:103C6000910548F09BC0209530952E0D3F1D283CB6
:103C7000310508F093C08F2F807F09F052C0E51303
:103C800014C0741312C0D62E61110FC0FF70F06102
:103C9000F093BB010E946E1D86EB91E00E94F1192A
:103CA0008091BB01F80185836CC1EF2831F05F3F43
:103CB00031F481E04F3F19F403C081E001C080E09E
:103CC00080FD03C081E0862701C080E0F82FF170FD
:103CD000FF2E80FF1CC0809184012091850136E079
:103CE000821709F428C190E0389FF001399FF00D48
:103CF0001124EA57FE4F7181571306C07081471394
:103D000003C07281671303C001968770E9CFD62E76
:103D1000662309F436C18091BB0181608093BB01A9
:103D200053C0E51308C0741306C0611104C0D80164
:103D30001596FC93AEC04D875E878D859E856A8BF8
:103D40000E94091D6A89882329F1D62E662311F164
:103D50002091BB01822F82958F7090E002970CF426
:103D600060C08091B6019091B70198878F831986C2
:103D7000FB86EA862C87CE01079651C0E51731F104
:103D80004D875E878D859E856A8B0E94091D6A8995
:103D900081112EC0C8010E94F119A4C08F2F807F0D
:103DA00069F77E2DF98AE88A89890E942E1D86EBA3
:103DB00091E00E94F119E6EBF1E086E0DF011D924F
:103DC0008A95E9F70E946E1DD12CDBC07413D8CF01
:103DD0006111D6CFD8011596FC93C8010E94F11944
:103DE000E6EBF1E086E0DF011D928A95E9F7C9C0B4
:103DF000D62E662379F22091BB01822F82958F7097
:103E000090E0029774F08091B6019091B7019A8387
:103E100089831B82FD82EC822E83CE0101960E9453
:103E2000F11986E0F801A6EBB1E001900D928A95B8
:103E3000E1F70E947C1D6FC0E216F30628F0C7016F
:103E4000821B930B9C0104C0209530952E0D3F1DC5
:103E5000283C310508F052C0D62E662309F49ACFCB
:103E6000E5132CC074132AC08091BB0180FD1DC0D6
:103E7000982F92959F70C9F0D80115968C9315973D
:103E80009F3039F09F5F9295907F8F70892B1596A8
:103E90008C93C8010E94F11986E0F801A6EBB1E00D
:103EA00001900D928A95E1F736C086E0F801A6EB05
:103EB000B1E001900D928A95E1F763C04D875E876E
:103EC0008D859E850E94091D882379F086E0F80182
:103ED000A6EBB1E001900D928A95E1F70E947C1D5E
:103EE0000E946E1DDD24D3944CC08091BB01816083
:103EF0008093BB01C8010E94F11943C07E2DF98A4D
:103F0000E88A89890E942E1DE6EBF1E086E0DF0158
:103F10001D928A95E9F70E946E1D33C0662309F44D
:103F200039CF4D875E878D859E850E94091D882328
:103F300009F430CFCBCF4D875E878D859E850E945B
:103F40002C22292F22952F7030E0223031052CF4BD
:103F50009F7041F0811106C00CC0243031052CF453
:103F60009F7049F4805E883020F0C8010E94F119EA
:103F7000CF2CDC2C06C0D80115969C91907F91F730
:103F8000F8CF8D2D62960FB6F894DEBF0FBECDBF71
:103F9000DF91CF911F910F91FF90EF90DF90CF9025
:103FA00008951F93CF93DF93CDB7DEB72C970FB64D
:103FB000F894DEBF0FBECDBF4F83588769877A87DD
:103FC0008B879C87CE0107960E94E41D8823C1F051
:103FD0002F8138858A859B85892B31F03F3F11F0F1
:103FE00080E003C02F3FE1F781E0811147C04F819E
:103FF000588569857A858B859C850E943D1D3EC0CC
:1040000086E0FE013796DE01119601900D928A95A9
:10401000E1F7FF81E8854A855B854115510531F05F
:10402000EF3F31F481E0FF3F19F403C081E001C0AC
:1040300080E080FD23C02091850130E0C901019618
:10404000877099276091840170E086179707F1F1D6
:10405000F983EA835D834C8396E0929FD001939F1E
:10406000B00D1124AA57BE4FFE01319601900D925A
:104070009A95E1F7809385010E944D1D16E080918D
:10408000840190918501891779F1189FC00111244D
:104090008A579E4F0E94E41D882331F1E0918401EC
:1040A0001E9FF0011124EA57FE4F40815181628129
:1040B0007381848195810E943D1D8091840190E0EF
:1040C00001968770992780938401D9CF0E94051D9E
:1040D0001092850110928401E6EBF1E086E0DF01A9
:1040E0001D928A95E9F7CACF2C960FB6F894DEBFD9
:1040F0000FBECDBFDF91CF911F910895EF92FF9238
:104100000F931F93CF93DF93FC01009709F46FC0C7
:10411000F12CEE24E394EF0121968491843740F44E
:10412000843008F055C0813081F0823021F15FC0C9
:10413000853709F447C0C0F19CE7980F903708F025
:1041400056C08F770E94941945C08F010E5F1F4F94
:10415000FE01849190E2980F983050F48770FE2D04
:1041600001C0FF0F8A95EAF78F2F0E94212315C007
:104170000E94CC1814C08F010E5F1F4FFE01849166
:1041800090E2980F983068F48770FE2D01C0FF0F01
:104190008A95EAF78F2F0E9427230E944A23E8017D
:1041A00019C00E949419FBCFCF010296FE01C49161
:1041B000CC2361F0EFE9FFE03197F1F700C0000098
:1041C000C150F6CFCF010296FE01F490EC0102C07F
:1041D0000E94CC188F2D882341F0EFE9FFE0319742
:1041E000F1F700C000008150F6CFFE0194CFDF91BF
:1041F000CF911F910F91FF90EF90089508956093D4
:10420000C0017093C1018093C2019093C3010C94CB
:10421000F31C0F931F930091C0011091C1012091D5
:10422000C2013091C301062B172B282B392B009389
:10423000C0011093C1012093C2013093C3011F91AB
:104240000F910C94F31C0F931F930091C0011091D8
:10425000C1012091C2013091C301062317232823F5
:1042600039230093C0011093C1012093C201309300
:10427000C3011F910F910C94F31C0F931F93009196
:10428000C0011091C1012091C2013091C3010627E4
:104290001727282739270093C0011093C1012093C5
:1042A000C2013093C3011F910F910C94F31C109223
:1042B000BC011092BD011092BE011092BF010C947E
:1042C000F31C41E050E060E070E004C0440F551F73
:1042D000661F771F8A95D2F74093BC015093BD01AA
:1042E0006093BE017093BF010C94F31C41E050E059
:1042F00060E070E004C0440F551F661F771F8A9569
:10430000D2F78091BC019091BD01A091BE01B09106
:10431000BF01842B952BA62BB72B8093BC019093C8
:10432000BD01A093BE01B093BF010C94F31C41E00A
:1043300050E060E070E004C0440F551F661F771F17
:104340008A95D2F740955095609570958091BC0103
:104350009091BD01A091BE01B091BF01842395232E
:10436000A623B7238093BC019093BD01A093BE0107
:10437000B093BF010C94F31C41E050E060E070E0AA
:1043800004C0440F551F661F771F8A95D2F780918E
:10439000BC019091BD01A091BE01B091BF018427E5
:1043A0009527A627B7278093BC019093BD01A093C2
:1043B000BE01B093BF010C94F31C0F931F930091A7
:1043C000BC011091BD012091BE013091BF01062BAF
:1043D000172B282B392B0093BC011093BD01209380
:1043E000BE013093BF011F910F910C94F31C0F93EA
:1043F0001F930091BC011091BD012091BE0130912D
:10440000BF0106231723282339230093BC011093EF
:10441000BD012093BE013093BF011F910F910C94F9
:10442000F31C0F931F930091BC011091BD012091CB
:10443000BE013091BF01062717272827392700938F
:10444000BC011093BD012093BE013093BF011F91A9
:104450000F910C94F31C0895CF92DF92EF92FF928C
:104460000F931F93CF93DF93EC01C090C001D090C6
:10447000C101E090C201F090C3018091BC01909114
:10448000BD01A091BE01B091BF01C82AD92AEA2A74
:10449000FB2A0FE110E0B701A601002E04C07695BB
:1044A0006795579547950A94D2F740FF07C0BE011C
:1044B000802F0E94420E8130910539F4015011097C
:1044C00050F7BE0180E00E94420EDF91CF911F9114
:1044D0000F91FF90EF90DF90CF90089590910C0195
:1044E000992361F190910D01992341F1982F9695AF
:1044F000969596959F3088F4E0910E01F0910F010A
:10450000E90FF11D877021E030E001C0220F8A958C
:10451000EAF78181822B818308959091D70190FFE2
:104520002DC01F928F9386E79AE09F938F930E94EE
:104530003F0A0F900F900F900F90089540910E0139
:1045400050910F0120E030E09FEFFA01E20FF31FDE
:104550006281681799F09F3F19F4611101C0922F91
:104560002F5F3F4F2E30310581F79F3F39F0FA0121
:10457000E90FF11D97FDFA958283089508959091B2
:104580000C01992369F190910D01992349F1982F1C
:104590009695969596959F3090F4E0910E01F09146
:1045A0000F01E90FF11D877021E030E001C0220FFB
:1045B0008A95EAF720958181282321830895909197
:1045C000D70190FF1FC01F928F9388E59AE09F93B9
:1045D0008F930E943F0A0F900F900F900F900895B5
:1045E00040910E0150910F0120E030E0FA01E20FFE
:1045F000F31F9281981301C012822F5F3F4F2E301C
:104600003105A1F7089581E090E0E0910E01F0916D
:104610000F01E80FF91F1082019680319105A9F76B
:1046200008959091D601982B9093D6010895809586
:104630009091D60198239093D60108951092D601B7
:1046400008959091D501982B9093D5010895809568
:104650009091D50198239093D50108951092D5019A
:1046600008958093C40108951092C4010895409163
:104670000E0150910F0120E030E080E0FA01E20FDE
:10468000F31F918191118F5F2F5F3F4F2F303105C5
:10469000A9F70895E0910E01F0910F018091D601E4
:1046A0008083E0910E01F0910F0180819091D501FE
:1046B000892B80839091C401992361F0E0910E01D0
:1046C000F0910F018081892B80830E943723811113
:1046D0001092C40180910E0190910F010C944E171D
:1046E00090933B0180933A0108958295982F9C7C8A
:1046F00096959695837344E0849F90011124922BA4
:10470000892F8A7A86959575990F892B08951F931D
:10471000CF93DF931F92CDB7DEB799830E947523A5
:10472000182F9981892F0E947523212F30E0322F75
:104730002227A901482BCA010F90DF91CF911F9129
:1047400008958091F001843009F11092D80120E49D
:1047500088E190E00FB6F894A895809360000FBEB2
:104760002093600083B7817F846083BF83B78160BB
:1047700083BF7894889583B78E7F83BF88E10FB617
:10478000F89480936000109260000FBE0895089521
:104790000895CF930E94C7230E94E80B0E94C8236C
:1047A000C0E08C2F0E94130D811105C0CF5FCE3069
:1047B000C1F780E001C081E0CF9108950C94051D00
:1047C00082E084BD93E095BD9AEF97BD80936E0023
:1047D00008952FB7F8948091D9019091DA01A091B2
:1047E000DB01B091DC012FBF0895CF92DF92EF92F1
:1047F000FF920F931F932FB7F8944091D9015091D6
:10480000DA016091DB017091DC012FBF6A017B014D
:10481000EE24FF248C0120E030E0C016D106E20631
:10482000F30610F441505109481B590BCA011F915E
:104830000F91FF90EF90DF90CF9008951F920F920D
:104840000FB60F9211248F939F93AF93BF938091D4
:10485000D9019091DA01A091DB01B091DC010196C0
:10486000A11DB11D8093D9019093DA01A093DB01C2
:10487000B093DC01BF91AF919F918F910F900FBECC
:104880000F901F9018950E944914F8942FEF87EA13
:1048900091E6215080409040E1F700C0000087E0A1
:1048A00090EBDC018093F9019093FA01A093FB0156
:1048B000B093FC012CE088E190E00FB6F894A89545
:1048C000809360000FBE20936000FFCFEF92FF92B5
:1048D0000F931F93CF93DF93E82EF12C8F2D0E941F
:1048E000130DC0E0D0E0082F10E098010C2E02C09C
:1048F000359527950A94E2F720FD05C02196C6302C
:10490000D10599F709C06C2F7F2D80E00E94200E01
:10491000E812F4CF81E005C0F3948EE0F812DECF08
:1049200080E0DF91CF911F910F91FF90EF9008955C
:10493000CF93C82F8CE20E946624882321F08C2F0D
:10494000CF910C94662480E0CF910895CF930E947C
:10495000F325811102C00E94D9258BE99AE00E94BB
:10496000A609C5E6C15049F00E94E80B8FE39CE917
:104970000197F1F700C00000F5CF84E99AE00E94AA
:10498000A60989E20E949824811111C18AE20E943D
:10499000982481110E94D92585E00E9498248111D4
:1049A0000E9443240E94FE258093D70187E00E9445
:1049B0009824882399F18BE10E949824882351F050
:1049C0009091D70191FB882780F921E0822780FB15
:1049D00091F922C08EE00E949824882351F0909192
:1049E000D70192FB882780F921E0822780FB92F98A
:1049F00013C080E10E9498249091D701882341F050
:104A000093FB882780F921E0822780FB93F904C07B
:104A1000892F809580FB90F99093D7018091D701E1
:104A20000E9402260E9410268093EA0180EE0E94D6
:104A30009824882341F08091EA01982F909590FB6B
:104A400080F98093EA0189E30E949824882359F031
:104A50009091EA0191FB882780F921E0822780FB71
:104A600091F99093EA0182EE0E949824882359F0EC
:104A70009091EA0192FB882780F921E0822780FB50
:104A800092F99093EA0186EE0E949824882359F0C7
:104A90009091EA0193FB882780F921E0822780FB2F
:104AA00093F99093EA0183EE0E949824882359F0A9
:104AB0009091EA0194FB882780F921E0822780FB0E
:104AC00094F99093EA0185E30E949824882359F091
:104AD0009091EA0195FB882780F921E0822780FBED
:104AE00095F99093EA0181E30E949824882359F074
:104AF0009091EA0196FB882780F921E0822780FBCC
:104B000096F99093EA0181E10E949824882359F054
:104B10009091EA0197FB882780F921E0822780FBAA
:104B200097F99093EA018091EA010E9414268091FE
:104B3000EA0187FB882780F980930D0187E20E94B4
:104B40009824C82F8EE10E9498248111C2608FE1C1
:104B50000E9498248111C46080E20E9498248111EF
:104B6000C86081E20E9498248111C06182E20E94A3
:104B700098248111C06283E20E9498248111C0644C
:104B800084E20E949824882311F0C06802C0CC23DC
:104B900029F08C2F0E940B266C2F03C00E94072641
:104BA000682F70E080E090E0CF910C94FF20CF91CF
:104BB00008956DEE7EEF80E090E00E94CE2F60E0E1
:104BC00082E090E00E94C02F60E083E090E00E94CD
:104BD000C02F60E084E090E00E94C02F60E085E09C
:104BE00090E00C94C02F80E090E00E94BA2F21E06A
:104BF0008D3E9E4F09F020E0822F089582E090E0E4
:104C00000C94B22F682F82E090E00C94C02F83E0C8
:104C100090E00C94B22F682F83E090E00C94C02FAA
:104C200084E090E00C94B22F682F84E090E00C9424
:104C3000C02F8091DF0180FF0BC06091130185E0E0
:104C4000689FB001112475956795759567952AC081
:104C500081FF09C06091130185E0689FB0011124B4
:104C6000759567951FC082FF07C06091130185E0AD
:104C7000689FB001112416C04091E0014423C9F09F
:104C800060911201461788F72091130185E0289F53
:104C900090011124429FC001439F900D112470E0A8
:104CA0000E94842F6038710540F46115710539F058
:104CB00002C065E070E0862F08958FE7089581E0D7
:104CC00008958091DF0180FF08C06091110170E0BC
:104CD000759567957595679521C081FF06C06091B0
:104CE000110170E07595679519C082FF04C060914D
:104CF000110170E010C08091E0018823C1F0609143
:104D000010018617A0F790911101989FC0011124FE
:104D100070E00E94842F6038710528F461157105D8
:104D200021F0862F08958FE7089581E0089561E0CE
:104D300070E0F4CF803F21F40E941926819504C0D1
:104D4000813F29F40E9419268093E3010895823F50
:104D500021F40E941926819504C0833F29F40E9402
:104D600019268093E2010895893F19F40E94612673
:104D700005C08A3F31F40E94612681958093E40149
:104D800008958B3F21F40E946126819504C08C3FD9
:104D900029F40E9461268093E5010895843F21F45F
:104DA0008091E101816017C0853F21F48091E1018C
:104DB000826011C0863F21F48091E10184600BC0C4
:104DC000873F21F48091E101886005C0883F31F47C
:104DD0008091E10180618093E10108958D3F21F48C
:104DE0008091DF0181600BC08E3F21F48091DF0153
:104DF000826005C08F3F29F48091DF018460809339
:104E0000DF010895803F39F48091E30187FF6CC092
:104E10001092E30169C0813F29F48091E3011816E3
:104E2000BCF362C09091E201823F29F497FF5CC01D
:104E30001092E20159C0833F19F41916CCF354C003
:104E4000893F41F48091E40118160CF04DC0109296
:104E5000E4014AC08A3F29F48091E40187FF44C0FD
:104E6000F6CF8B3F39F48091E50187FF3DC010926A
:104E7000E5013AC08C3F29F48091E5011816BCF396
:104E800033C0843F21F48091E1018E7F17C0853FBC
:104E900021F48091E1018D7F11C0863F21F4809142
:104EA000E1018B7F0BC0873F21F48091E101877F77
:104EB00005C0883F31F48091E1018F7E8093E1014C
:104EC00013C08D3F21F48091DF018E7F0BC08E3F98
:104ED00021F48091DF018D7F05C08F3F29F48091FF
:104EE000DF018B7F8093DF018091E20181110EC091
:104EF0008091E30181110AC08091E401811106C013
:104F00008091E501811102C01092E0010895809125
:104F1000D70183FF7EC087ED9AE00E94A6098091A9
:104F2000E1011F928F9382ED9AE09F938F930E94ED
:104F30003F0A80ED9AE00E94A6092091E201822FAB
:104F4000992787FD90959F932F938DEC9AE09F93DF
:104F50008F930E943F0A8BEC9AE00E94A609209151
:104F6000E301822F992787FD90959F932F9388ECDB
:104F70009AE09F938F930E943F0A86EC9AE00E94EA
:104F8000A6092091E401822F992787FD90959F9390
:104F90002F9383EC9AE09F938F930E943F0A81ECBA
:104FA0009AE00E94A6092091E501822F992787FDAA
:104FB00090959F932F938EEB9AE09F938F930E94EF
:104FC0003F0A8BEB9AE00E94A6098091E0011F92B4
:104FD0008F9388EB9AE09F938F930E943F0A86EB12
:104FE0009AE00E94A6098091DF011F928F9383EBC4
:104FF0009AE09F938F930E943F0A80EB9AE00E9471
:10500000A6098DB79EB74C960FB6F8949EBF0FBEFB
:105010008DBF81EE91E00E9493170E94E923909347
:10502000DE018093DD0108951F93CF93DF9380917C
:10503000DD019091DE010E94F5234091E0014423BF
:1050400021F02091140130E006C0209115015AE0B2
:10505000259F900111248217930708F482C0809144
:10506000E2011091E301D091E401C091E5018111C9
:1050700007C0111105C0D11103C0CC2309F471C0C0
:105080004F3F19F04F5F4093E001181624F40E943F
:1050900019268093E2018091E20187FF05C00E94FA
:1050A000192681958093E201111624F40E94192695
:1050B0008093E3018091E30187FF05C00E941926D8
:1050C00081958093E3016091E201662339F11091AB
:1050D000E301112319F1772767FD7095872F972F2B
:1050E0000E94892E23E333E343E35FE30E94ED2E26
:1050F0000E94562E6093E201612F772767FD70951D
:10510000872F972F0E94892E23E333E343E35FE346
:105110000E94ED2E0E94562E6093E3011D1624F48A
:105120000E9461268093E4018091E40187FF05C01D
:105130000E94612681958093E4011C1624F40E944C
:1051400061268093E5018091E50187FF05C00E94FB
:10515000612681958093E501DF91CF911F910C9499
:105160008727DF91CF911F910895E1EEF1E085E06F
:10517000DF011D928A95E9F71092E0011092DF019C
:1051800008958AEF9CE00E94A6091F9281E08F9308
:105190001F9285E08F938CEA9CE09F938F930E94EF
:1051A0003F0A0F900F900F900F900F900F9008955F
:1051B0008330E9F128F4813061F0823009F10895FB
:1051C000853009F462C008F449C0863009F474C01F
:1051D000089520911501862F90E0820F911D8F3F39
:1051E000910520F4620F6093150103C08FEF809347
:1051F0001501809115011F928F9385EE9BE072C07F
:1052000020911401862F90E0820F911D8F3F910510
:1052100020F4620F6093140103C08FEF8093140198
:10522000809114011F928F9383ED9BE05BC02091CE
:105230001301862F90E0820F911D8F3F910520F47E
:10524000620F6093130103C08FEF8093130180916D
:1052500013011F928F9380EC9BE044C020911201B8
:10526000862F90E0820F911D8F3F910520F4620FF1
:105270006093120103C08FEF80931201809112019D
:105280001F928F938BEA9BE02DC020911101862FF6
:1052900090E0820F911D8F3F910520F4620F609383
:1052A000110103C08FEF80931101809111011F92B2
:1052B0008F9382E99BE016C020911001862F90E029
:1052C000820F911D8F3F910520F4620F60931001B2
:1052D00003C08FEF80931001809110011F928F9374
:1052E00087E79BE09F938F930E943F0A0F900F9058
:1052F0000F900F900895833081F128F4813059F098
:105300008230D1F00895853009F449C0B8F1863073
:1053100009F456C0089580911501681720F4861B82
:105320008093150102C010921501809115011F9202
:105330008F9388E69BE054C080911401681720F495
:10534000861B8093140102C01092140180911401F5
:105350001F928F9386E59BE043C0809113016817ED
:1053600020F4861B8093130102C0109213018091D8
:1053700013011F928F9383E49BE032C0809112014E
:10538000681720F4861B8093120102C0109212014C
:10539000809112011F928F938EE29BE021C0809139
:1053A0001101681720F4861B8093110102C010922E
:1053B0001101809111011F928F9385E19BE010C034
:1053C00080911001681720F4861B8093100102C0A1
:1053D00010921001809110011F928F938AEF9AE032
:1053E0009F938F930E943F0A0F900F900F900F9002
:1053F0000895CF93C82F1F928F932FEF3DE03F93D7
:105400002F930E943F0A61E070E080E090E004C0CA
:10541000660F771F881F991FCA95D2F70E94FF2039
:105420000F900F900F900F90CF910C94051DCF937C
:105430008D3109F465C0B0F58E3009F4CBC100F5AB
:10544000873009F49BC1A8F4863009F06AC28091C4
:10545000D701817F8E7F8093D70184E09EE00E94F8
:10546000A60989E492E10E94A60981E08093E70100
:1054700080C1883009F44FC08B3009F47CC151C21F
:10548000863109F4EDC138F4803109F4B6C18131B7
:1054900009F42DC246C2893109F4CBC18B3109F41C
:1054A00086C13FC2853309F434C248F4873209F417
:1054B00030C208F430C2893209F42BC232C28334BC
:1054C00038F48A3308F029C2883309F454C129C258
:1054D000833409F41EC2883409F023C20E94051DDA
:1054E00088E392E10E94A6099FEF23ED80E39150AB
:1054F00020408040E1F700C000000E94432439C1F1
:1055000088E592E10E94A6090E94102E0E9442178F
:105510000E94800F2EC18DE492E10E94A60985E1D0
:1055200090E10E94A6090E9407261F928F9382E1B4
:1055300090E19F938F930E943F0A80E190E10E9447
:10554000A6090E94FE25C82F8DEF9FE00E94A609A4
:105550001F92CF9328EF3FE03F932F930E943F0A83
:1055600086EF9FE00E94A6098CEE9FE00E94A609AC
:105570008C2F81701F928F9329EE3FE03F932F93E2
:105580000E943F0A87EE9FE00E94A6098DED9FE0F2
:105590000E94A609C1FB882780F91F928F932AEDEC
:1055A0003FE03F932F930E943F0A88ED9FE00E94C7
:1055B000A6098CEC9FE00E94A609C2FB882780F90F
:1055C0001F928F9329EC3FE03F932F930E943F0A55
:1055D00087EC9FE00E94A6098EEB9FE00E94A6093F
:1055E000C3FBCC27C0F91F92CF938BEB9FE09F9317
:1055F0008F930E943F0A89EB9FE00E94A6090E94B8
:105600001026C82F85EA9FE00E94A6091F92CF931B
:1056100020EA3FE03F932F930E943F0A8EE99FE0EC
:105620000E94A60985E89FE00E94A6098C2F817040
:105630001F928F9322E83FE03F932F930E943F0AEF
:105640008DB79EB780960FB6F8949EBF0FBE8DBFE4
:1056500080E89FE00E94A60989E69FE00E94A609D3
:10566000C1FB882780F91F928F9326E63FE03F9386
:105670002F930E943F0A84E69FE00E94A60982E5DC
:105680009FE00E94A609C2FB882780F91F928F9392
:105690002FE43FE03F932F930E943F0A8DE49FE069
:1056A0000E94A6098BE39FE00E94A609C3FB8827FE
:1056B00080F91F928F9328E33FE03F932F930E943E
:1056C0003F0A86E39FE00E94A6098CE29FE00E94C9
:1056D000A609C4FB882780F91F928F9329E23FE037
:1056E0003F932F930E943F0A87E29FE00E94A60902
:1056F00085E19FE00E94A609C5FB882780F91F92DB
:105700008F9322E13FE03F932F930E943F0A80E175
:105710009FE00E94A60984EF9EE00E94A609C6FBB6
:10572000882780F91F928F9321EF3EE03F932F93BC
:105730000E943F0A8FEE9EE00E94A60987EE9EE03F
:105740000E94A609C7FBCC27C0F91F92CF9384EE15
:105750009EE09F938F930E943F0A82EE9EE00E94FC
:10576000A6098DB79EB74C960FB6F8949EBF0FBE94
:105770008DBFC1E0DBC08BE29EE058C08091D701B5
:10578000C82FC17080FF09C08BE292E10E94A60978
:105790008091D701817F8E7F44C08FE192E10E948A
:1057A000A6098091D70181608093D701E2CF8091D3
:1057B000D70181FBCC27C0F991E0C927C0FB81F953
:1057C0008093D701CC2319F082E192E125C084E0D7
:1057D00092E12CC08091D70182FBCC27C0F991E0E7
:1057E000C927C0FB82F98093D701CC2319F085EF3C
:1057F00091E112C085EE91E119C08091D70183FB40
:10580000CC27C0F991E0C927C0FB83F98093D70169
:10581000CC2351F089ED91E10E94A6098091D70136
:1058200081608093D70182C08CEC91E10E94A6092F
:10583000A0CF8DEB91E10E94A60981E991E10E9440
:10584000A60984E591E10E94A60987E291E10E9400
:10585000A60983EE90E10E94A60985EB90E1E6CFD0
:1058600087EA90E10E94A6090E9442171F928F9337
:105870008DE890E19F938F930E943F0A80910C01E5
:105880001F928F9386E790E19F938F930E943F0A28
:1058900080916E011F928F9383E690E19F938F9387
:1058A0000E943F0A80910D011F928F9380E590E145
:1058B0009F938F930E943F0A8091D9019091DA01C2
:1058C000A091DB01B091DC01BF93AF939F938F93C5
:1058D0008CE390E19F938F930E943F0A8DB79EB710
:1058E00046960FB6F8949EBF0FBE8DBF42CF0E9462
:1058F000051DC0910D0181E0C827C0930D01CC2387
:1059000029F082E390E10E94A60910C087E290E1AD
:105910008DCF80E003C08D5101C089530E94F929C9
:1059200028CF85E290E10E94A609C0E08C2FCF919C
:10593000089580E0089580E00895CF93C82F809166
:10594000E701813081F020F0823009F44CC042C17F
:10595000A0910E01B0910F018C91813169F08232DA
:1059600009F03AC109C0A0910E01B0910F018C91CC
:10597000813111F0823249F48C2F0E94992C8111CF
:105980002FC08C2F0E94172A2CC08C2F0E949B2C7A
:10599000811126C0C431E1F070F4CB3081F0C03108
:1059A000D1F40E94C12887EF9DE00E94A60982E001
:1059B0008093E70115C0C93259F0C83361F484E01F
:1059C0009EE00E94A6098BEF9DE00E94A60908C0F8
:1059D0001092E70103C185EF9DE00E94A609FEC079
:1059E00081E08170FDC0C43220F5CE3108F0C0C026
:1059F000CB3099F1C8F4C73009F0D2C08AE0809367
:105A0000150194E19093140193E090931301809316
:105A1000120188E08093110188E2809310018BE9E4
:105A20009CE00E94A609BFC0C33149F1C431C1F056
:105A3000B7C0CB3409F4A9C028F4C93289F0C833FF
:105A400061F0AEC0C13509F49EC0C23509F499C0F9
:105A5000CE3409F0A5C06AE09EC00E94C128A3C050
:105A60008091E601882319F01092E6019CC088EA33
:105A70009CE00E94A60981E08093E701B1C082E822
:105A80009CE00E94A60980E79CE00E94A609809104
:105A900015011F928F938DE69CE09F938F930E9438
:105AA0003F0A8BE69CE00E94A60989E59CE00E94E3
:105AB000A609809114011F928F9386E59CE09F9325
:105AC0008F930E943F0A84E59CE00E94A60985E42A
:105AD0009CE00E94A609809113011F928F9382E49B
:105AE0009CE09F938F930E943F0A80E49CE00E9479
:105AF000A6098FE29CE00E94A609809112011F92E4
:105B00008F938CE29CE09F938F930E943F0A8AE2DE
:105B10009CE00E94A60985E19CE00E94A609809174
:105B200011011F928F9382E19CE09F938F930E94BB
:105B30003F0A80E19CE00E94A60989EF9BE00E9459
:105B4000A609809110011F928F9386EF9BE09F938F
:105B50008F930E943F0A84EF9BE00E94A6098DB7B5
:105B60009EB748960FB6F8949EBF0FBE8DBF1BC060
:105B7000CE51EC2FF0E0E15DFE4F80818093E60195
:105B800012C061E003C061E006C06AE08091E601F6
:105B90000E94D82808C08091E6010E947B2903C09A
:105BA00089E99CE013C08091E601882369F01F9287
:105BB0008F9383E99CE09F938F930E943F0A0F90FD
:105BC0000F900F900F9004C080E99CE00E94A609FE
:105BD00081E006C01092E70180E002C080E001CFC2
:105BE000CF910895E1E8F0E0808188608083808132
:105BF000816080838FB7F89493E09093890090ED53
:105C0000909388008FBF0895EFE6F0E08081826076
:105C100080830895EFE6F0E080818D7F8083089592
:105C2000EFE6F0E0808192E08927808308951F925B
:105C30000F920FB60F9211242F933F934F935F93C0
:105C40006F937F938F939F93AF93BF93EF93FF9344
:105C50008091E8019091E90101969093E901809388
:105C6000E801811103C082E00E94800FE091E90108
:105C7000E695E695F0E0E859FD4EE4918091E80163
:105C80008E1303C080E00E94800FFF91EF91BF91BF
:105C9000AF919F918F917F916F915F914F913F91C4
:105CA0002F910F900FBE0F901F90189504D06894FD
:105CB000B1118DC0089570D088F09F5790F0B92F22
:105CC0009927B751A0F0D1F0660F771F881F991F51
:105CD0001AF0BA95C9F712C0B13081F077D0B1E0AF
:105CE000089574C0672F782F8827B85F39F0B93FBF
:105CF000CCF3869577956795B395D9F73EF4909553
:105D00008095709561957F4F8F4F9F4F0895E894D0
:105D100009C097FB3EF490958095709561957F4FF3
:105D20008F4F9F4F9923A9F0F92F96E9BB279395A1
:105D3000F695879577956795B795F111F8CFFAF4B1
:105D4000BB0F11F460FF1BC06F5F7F4F8F4F9F4FE2
:105D500016C0882311F096E911C0772321F09EE840
:105D6000872F762F05C0662371F096E8862F70E0A6
:105D700060E02AF09A95660F771F881FDAF7880F80
:105D80009695879597F9089557FD9058440F551F9C
:105D900059F05F3F71F04795880F97FB991F61F0AD
:105DA0009F3F79F087950895121613061406551F24
:105DB000F2CF4695F1DF08C0161617061806991F90
:105DC000F1CF86957105610508940895E894BB2785
:105DD00066277727CB0197F908950BD078C069D053
:105DE00028F06ED018F0952309F05AC05FC0112436
:105DF000EECFCADFA0F3959FD1F3950F50E0551F6A
:105E0000629FF001729FBB27F00DB11D639FAA270F
:105E1000F00DB11DAA1F649F6627B00DA11D661F5E
:105E2000829F2227B00DA11D621F739FB00DA11D7F
:105E3000621F839FA00D611D221F749F3327A00D39
:105E4000611D231F849F600D211D822F762F6A2FD5
:105E500011249F5750408AF0E1F088234AF0EE0F5A
:105E6000FF1FBB1F661F771F881F91505040A9F767
:105E70009E3F510570F014C0AACF5F3FECF3983EEF
:105E8000DCF3869577956795B795F795E7959F5FCE
:105E9000C1F7FE2B880F911D9695879597F9089568
:105EA00097F99F6780E870E060E008959FEF80ECCD
:105EB000089500240A941616170618060906089570
:105EC00000240A9412161306140605060895092ED6
:105ED0000394000C11F4882352F0BB0F40F4BF2B45
:105EE00011F460FF04C06F5F7F4F8F4F9F4F089585
:105EF000991B79E004C0991F961708F0961B881F1C
:105F00007A95C9F78095089597FB072E16F40094AB
:105F100007D077FD09D00E949E2F07FC05D03EF4E4
:105F2000909581959F4F0895709561957F4F089545
:105F3000EE0FFF1F0590F491E02D0994AA1BBB1BE7
:105F400051E107C0AA1FBB1FA617B70710F0A61B79
:105F5000B70B881F991F5A95A9F780959095BC019A
:105F6000CD010895F999FECF92BD81BDF89A992788
:105F700080B50895A8E1B0E042E050E00C94D52F40
:105F8000262FF999FECF1FBA92BD81BD20BD0FB655
:105F9000F894FA9AF99A0FBE019608950E94C02FBC
:105FA000272F0C94C12FDC01CB01FC01F999FECF06
:105FB00006C0F2BDE1BDF89A319600B40D92415091
:0A5FC0005040B8F70895F894FFCFA1
:105FCA002002810F72104F101B10E80F0101C5014A
:105FDA0028080A03140A3F4D362039E50998096250
:105FEA0009420909097C089508AE08C708E70801AB
:0A5FFA000203040506070809000071
:00000001FF
